:020000040800F2
:1000000000070020E5040008E91300086913000850
:10001000C11300086913000895130008E7040008DD
:10002000E7040008E7040008E70400080D390008A9
:10003000E7040008E7040008E7040008E7040008F4
:10004000E7040008E7040008E7040008E7040008E4
:10005000E7040008E7040008393D0008653D000892
:10006000913D0008BD3D0008E93D0008E704000897
:10007000E7040008E7040008E7040008E7040008B4
:10008000E7040008E7040008E7040008E526000884
:1000900051270008A5270008F9270008153E000889
:1000A000E7040008E7040008E7040008E704000884
:1000B000893B0008E7040008E7040008E70400089B
:1000C000E7040008E7040008E7040008E704000864
:1000D000E7040008E7040008912A0008E704000884
:1000E0007D3E0008E7040008E7040008E704000874
:1000F000E7040008E7040008E7040008E704000834
:10010000E7040008E7040008E7040008E704000823
:10011000E7040008E7040008E7040008E704000813
:10012000E7040008E7040008E7040008E704000803
:10013000E7040008E7040008E7040008E7040008F3
:10014000E7040008E7040008E7040008E7040008E3
:10015000E7040008E7040008E7040008E7040008D3
:10016000E7040008E7040008E7040008E7040008C3
:10017000E7040008E7040008E7040008E7040008B3
:10018000E7040008E7040008E7040008E7040008A3
:10019000E7040008E7040008E7040008E704000893
:1001A000E7040008E7040008E7040008E704000883
:1001B000E7040008E7040008E7040008E704000873
:1001C000E7040008E7040008E7040008E704000863
:1001D000E7040008E7040008E7040008E704000853
:1001E00053B94AB9002908BF00281CBF4FF0FF319E
:1001F0004FF0FF3000F074B9ADF1080C6DE904CE9A
:1002000000F006F8DDF804E0DDE9022304B07047F1
:100210002DE9F047089D04468E46002B4DD18A42B9
:10022000944669D9B2FA82F252B101FA02F3C2F1EC
:10023000200120FA01F10CFA02FC41EA030E94407D
:100240004FEA1C48210CBEFBF8F61FFA8CF708FB9E
:1002500016E341EA034306FB07F199420AD91CEB76
:10026000030306F1FF3080F01F81994240F21C81A8
:10027000023E63445B1AA4B2B3FBF8F008FB1033F0
:1002800044EA034400FB07F7A7420AD91CEB040425
:1002900000F1FF3380F00A81A74240F207816444F5
:1002A000023840EA0640E41B00261DB1D44000237A
:1002B000C5E900433146BDE8F0878B4209D9002DDE
:1002C00000F0EF800026C5E9000130463146BDE868
:1002D000F087B3FA83F6002E4AD18B4202D38242D2
:1002E00000F2F980841A61EB030301209E46002D81
:1002F000E0D0C5E9004EDDE702B9FFDEB2FA82F2D6
:10030000002A40F09280A1EB0C014FEA1C471FFA33
:100310008CFE0126200CB1FBF7F307FB131140EA1A
:1003200001410EFB03F0884208D91CEB010103F1E7
:10033000FF3802D2884200F2CB804346091AA4B2A9
:10034000B1FBF7F007FB101144EA01440EFB00FE7D
:10035000A64508D91CEB040400F1FF3102D2A645E2
:1003600000F2BB800846A4EB0E0440EA03409CE781
:10037000C6F12007B34022FA07FC4CEA030C20FA2E
:1003800007F401FA06F31C43F9404FEA1C4900FA4E
:1003900006F3B1FBF9F8200C1FFA8CFE09FB1811CB
:1003A00040EA014108FB0EF0884202FA06F20BD93E
:1003B0001CEB010108F1FF3A80F08880884240F28E
:1003C0008580A8F102086144091AA4B2B1FBF9F0D2
:1003D00009FB101144EA014100FB0EFE8E4508D9CD
:1003E0001CEB010100F1FF346CD28E456AD9023852
:1003F000614440EA0840A0FB0294A1EB0E01A14237
:10040000C846A64656D353D05DB1B3EB080261EBA4
:100410000E0101FA07F722FA06F3F1401F43C5E97E
:10042000007100263146BDE8F087C2F12003D840B4
:100430000CFA02FC21FA03F3914001434FEA1C47F6
:100440001FFA8CFEB3FBF7F007FB10360B0C43EAE8
:10045000064300FB0EF69E4204FA02F408D91CEB98
:10046000030300F1FF382FD29E422DD90238634496
:100470009B1B89B2B3FBF7F607FB163341EA034136
:1004800006FB0EF38B4208D91CEB010106F1FF3885
:1004900016D28B4214D9023E6144C91A46EA00467C
:1004A00038E72E46284605E70646E3E61846F8E60E
:1004B0004B45A9D2B9EB020864EB0C0E0138A3E757
:1004C0004646EAE7204694E74046D1E7D0467BE738
:1004D000023B614432E7304609E76444023842E7B0
:1004E000704700BF02E000F000F8FEE772B63A483D
:1004F00080F30888394880F3098839484EF6085156
:10050000CEF20001086040F20000CCF200004EF68E
:100510003471CEF200010860BFF34F8FBFF36F8FCD
:1005200040F20000C0F2F0004EF68851CEF2000119
:100530000860BFF34F8FBFF36F8F4FF00000E1EE05
:10054000100A4EF63C71CEF200010860062080F3DE
:100550001488BFF36F8F03F059FA03F035FA03F0F4
:100560007FFA4FF055301F491B4A91423CBF41F87A
:10057000040BFAE71C49194A91423CBF41F8040BAD
:10058000FAE71A491A4A1B4B9A423EBF51F8040B2C
:1005900042F8040BF8E700201749184A91423CBF83
:1005A00041F8040BFAE703F013FA03F0A7FA144C2E
:1005B000144DAC4203DA54F8041B8847F9E700F005
:1005C00041F8114C114DAC4203DA54F8041B884732
:1005D000F9E703F0FBB9000000070020002300202A
:1005E000000000080001002000070020684100080A
:1005F000002300202423002028230020A0390020ED
:10060000E0010008E0010008E0010008E001000846
:100610002DE9F04F2DED108AC1F80CD0C3689D462E
:10062000BDEC108ABDE8F08F002383F311882846C3
:10063000A047002002F040FEFEE702F0C5FD00DF0B
:10064000FEE70000F8B503F0FFF8074603F04AF9AB
:10065000054600283FD12C4B9F423CD001339F429E
:100660003CD02A4B27F0FF029A423AD1F8B200F070
:1006700063FB2E4642F2107400F064FB08B10024C4
:10068000264600F0F9FF80B3032000F045F800246F
:10069000264635B11E4B9F4203D003F01BF90024C0
:1006A0002646002003F0DAF81A4B1B691B0422D4FB
:1006B0000EB100F047F800F0A3FB00F08BFD00F056
:1006C00095FE0546CCB100F091FE401BA04214D926
:1006D00000F038F8F3E72E460024CDE70446012663
:1006E000CAE706464FF47A74C6E7002CD1D04FF41F
:1006F0007A740126CDE70024DDE700F035FC4FF4E5
:100700007A7002F0DFFDDDE7010007B0000008B0FD
:10071000263A09B000040240084B187003280CD890
:10072000DFE800F008050208022000F0B5BD022055
:1007300000F0A8BD024B00225A6070472823002019
:100740002C23002010B500F097FF30B1204B03227E
:100750001A70204B00225A6010BD1F4B1F4A1C46C6
:1007600019680131F8D004339342F9D162681C4B07
:100770009A42F1D91B4B9B6803F1006303F5803368
:100780009A42E9D203F07AF803F08CF8002000F0E6
:100790003BFD0220FFF7C0FF134B1A6C00221A64C6
:1007A000196E1A66196E596C5A64596E5A665B6EE8
:1007B00072B64FF0E0232021C3F8084DD4E900328F
:1007C00081F311889D4683F308881047C4E700BF72
:1007D000282300202C23002000000108200001080D
:1007E000FFFF00080023002000380240094A136878
:1007F00049F2690099B21B0C00FB01331360064BF0
:10080000186844F2506182B2000C01FB02001860CB
:1008100080B27047202300201C23002010B5002147
:100820001022044600F054FD034B03CB20606160AE
:100830001868A06010BD00BF107AFF1F2DE9F041BD
:10084000ADF54E7D0DF134086CAC40F275120746E3
:100850000D460EA80021C8F8001000F039FD4FF435
:10086000C4720021204600F033FD00F0BFFD254B8F
:100870004FF47A72B0FBF2F0186093E8070001239E
:1008800084E807000DF5E9702382FFF7C7FF4FF4F6
:10089000A4431D49238406A803F09AFB192384F876
:1008A00032310DF2E32206AB0DF1300C1E4603CEC1
:1008B000664510605160334602F10802F6D1337884
:1008C000137041460122204600F094FD002303935B
:1008D000AB7E029305F11903019380B20123CDE9A8
:1008E00004800093E97E05A3D3E90023384601F094
:1008F00017FA0DF54E7DBDE8F08100BF9E6AC42158
:10090000818A46EE34230020E03F00082DE9F043C1
:10091000224DBBB000F06AFDAB6840F2ED22C31A75
:10092000934232D906AFA8602B46282200213846D0
:1009300001F0DEFB05F10E0000F0C2FC00260446CB
:100940005FFA80F905F10E08F3B2F100994501F163
:10095000280107D908EB06030822384601F0C8FB36
:100960000136F1E708230122CDE9023205340C4BB0
:100970000193A4B230230093CDE9047405A3D3E915
:100980000023297B074801F0CBF93BB0BDE8F08399
:10099000AFF3008078F6339F93CACD8D7833002073
:1009A000853300204C330020F0B58B8A013B9BB28D
:1009B000C92BC9B006460C4647D8274D2F7B27BB0D
:1009C00005F10C03009308223B463946204601F00E
:1009D00053FA7B1CFAB2D9001F46A38A013B9A4204
:1009E00005DA0E322A44009200230822EEE70023A3
:1009F0000022C5E900230023AB6085F8D730C5F895
:100A0000D8302B7B0BB9E37E2B738122002106ADFE
:100A100027A800F05DFC0122294627A800F0B8FDB8
:100A200000230393A37E029304F1190380B2019380
:100A30002823CDE90450E17E0093304604A3D3E996
:100A4000002301F06DF9FFF761FF49B0F0BD00BF71
:100A500026417272DF25D7B77833002070B50D4676
:100A600014461E4601F0F2F850B9022E10D1012CA6
:100A70000ED112A3D3E90023C5E90023012007E02A
:100A8000282C10D005D8012C09D0052C0FD000201F
:100A900070BD302CFBD10BA3D3E90023ECE70BA3F3
:100AA000D3E90023E8E70BA3D3E90023E4E70BA392
:100AB000D3E90023E0E700BFAFF30080401DA12091
:100AC00026812A0B78F6339F93CACD8D9E6AC42166
:100AD000818A46EE26417272DF25D7B7F017304A79
:100AE00039059E562DE9F04F8DB002AF80460D4678
:100AF00001F0ACF8044600285CD12B7E022B1BD100
:100B0000EB8A012B18D100F071FC0646FFF76EFE50
:100B100003464FF4C870DFF81C92B3FBF0F206F501
:100B2000167602FB103316FA83F3C9F80030EB7E19
:100B300033B97B4B00221A702C37BD46BDE8F08FCD
:100B4000AB8AE6B2013BB34204F101040CD907F1D0
:100B500008031E44E10000960023082201F0F8017A
:100B6000284601F089F9EBE707F11800FFF756FE78
:100B7000324607F1180107F1080003F0F7F90028E1
:100B8000D7D10F2E08D8664B1E70D9F80030A3F5C8
:100B90001673C9F80030CFE7FB1DF87101460093CA
:100BA00007220346284601F067F9F979404601F02B
:100BB00045F8C1E7EB8A282B26D010D8012B1ED090
:100BC000052BB9D1BFF34F8F5649574BCA6802F472
:100BD000E0621343CB60BFF34F8F00BFFDE7302BC4
:100BE000AAD16B7E514C0133627BDBB29342E94662
:100BF00003D1EA7E237B9A420BD0CD469CE729465F
:100C00004046FFF71BFE97E729464046FFF7CCFE1C
:100C100092E74FF0000807F11803A7F81880102298
:100C2000009341460123284601F026F9AE8A023E90
:100C3000B6B2F31C9B109B000733DB08A9EBC30380
:100C40009D460DF1080A1FFA88F34FEAC8019E423B
:100C500001F110010AD90AEB0803009308220023CE
:100C6000284601F009F908F10108ECE794F8D700EB
:100C700000F0D4FAD4F8D810054619B994F8D70082
:100C800000F0DCFAD4F8D83033449D4205D294F811
:100C9000D7000021013000F0D1FA4FEA960B4FF057
:100CA00000081FFA88F18B45D4E9003209D90AEB14
:100CB000880103EB8800012200F012FB08F1010813
:100CC000EFE7F31842F10002C4E90032D4F8D8305B
:100CD00094F8D70006EB0308C4F8D88000F09EFA19
:100CE000804509D394F8D730D4F8D8000133401B9D
:100CF00084F8D730C4F8D800FF2E0D4D09D8002352
:100D0000237300F0AFFA00F0B7FC288108B9FFF7B1
:100D100019FD23689B0A01332B810023A3606CE734
:100D20004533002000ED00E00400FA057833002090
:100D30003423002048330020014B1870704700BF57
:100D40004023002030B54FF00054244B22689A42D3
:100D500085B007D002F0D0FD0446A8B90024204693
:100D600005B030BD1E4B627D1A701E48237D037393
:100D70001D49C9220E3000F099FA2046E0220021D8
:100D800000F0A6FA0124EAE7184A194D136C43F063
:100D900000731364AA6D174B9A42DFD12B6E013B8F
:100DA0007E2BDBD8144A07CA01AB83E8070018463C
:100DB000032100F02FFC6B6D83424FF00003CDD177
:100DC0002A6D8A4201BFAB65054B2A6E1A7003BFBC
:100DD0000A4BEA6D1A601C46C1E700BF9AAD44C5D4
:100DE0004023002078330020160000200038024005
:100DF000006600405041A0B0586600401823002013
:100E00002DE9FF474C4C00F037FC022363710023AF
:100E100002934A4B2081D3F800C0BCF57A7F12D3ED
:100E2000474B484FB7FBFCF69C458CBF0A23112368
:100E3000581EB6FBF3F503FB1562C1B2002A3ED083
:100E400002280346F4D89DF80B303F493F485A1E0C
:100E50009DF80A30013B1B0443EA0253BDF8082009
:100E6000013A13434B6001F0CFFE00230193384B4E
:100E7000384900933848394B4FF4805200F0B8FE9F
:100E8000374B197811B1344800F0D8FE00F0AEFAB3
:100E90000546FFF7ABFC4FF4C873B0FBF3F202FB5F
:100EA000130305F5167010FA83F02E4B186002F04C
:100EB00019FD08B10F23238104B0BDE8F0876B1E34
:100EC000B3F5806FBFD2C1EBC10E0EF103034FEA41
:100ED000E309C3F3C703A1EB030809F1010A4FF4C7
:100EE0007A705FFA88F609FB00005AFA88F8B0FBBE
:100EF000F8F0B0F5617F08D90EF1FF33C3F3C703F3
:100F0000C91ACEB2591E0F2914D8721E072A8CBFD7
:100F100000220122991901FB0551B7FBF1F7BC45ED
:100F200091D1002A8FD0ADF808508DF80A308DF895
:100F30000B6088E71346EDE73423002018230020D8
:100F40003F420F0040787D011023002090340020A4
:100F50005D0A0008442300204C330020E50A000805
:100F600040230020483300202DE9F04F91A7D7E916
:100F700000670FF24829D9E90089874D93B0DFF85F
:100F800044B2864C284600F02FFF0DF1300A07903E
:100F900070B310220021504600F09AF9079B197B8C
:100FA0004FF0000261F303028DF830205868996811
:100FB0000EAA03C21B680D9A63F31C029DF8303021
:100FC0000D9243F020038DF830300023524619462D
:100FD000584601F029FE079028B9284600F008FF7E
:100FE000079B2370CEE72378072B3CD8013323706F
:100FF00018220021504600F06BF9DFF8C8B1684CA8
:10100000002319465246584601F036FE014670BB91
:10101000102208A800F05CF9636983F480636361BF
:1010200000F0E6F90B4612A9024611E903000DF1A2
:10103000240C8CE803009DF83410C1F303008906EA
:101040004CBF0E99BDF838C08DF82C0046BFC1F3D7
:101050001C0C4CF00041CCF30A010891284608A969
:1010600001F08EF8CCE7284600F0C2FEC0E7284623
:1010700000F0ECFD0446002848D1DFF84CB100F048
:10108000B5F9DBF80030984240D300F0AFF9079093
:10109000FFF7ACFB079A8DF8204003464FF4C87069
:1010A00002F51672B3FBF0F101FB103312FA83F371
:1010B000CBF80030DFF814B19BF8001011B9012310
:1010C0008DF8203050460791FFF7A8FB0799C1F132
:1010D0001004E4B2062C28BF0624224651440DF128
:1010E000210000F0E3F808AB0393182302930134C6
:1010F0002C4B0193E4B20123009304943B46324607
:10110000284600F0A5FD00238BF8003000F06EF9B2
:10111000254A264C1368C31AB3F57A7F30D3106082
:1011200000F066F902460B46284600F06BFE2846A2
:1011300000F08CFD20B3237BDFF894B0002B14BFAC
:10114000032302238BF8053000F050F94FF47A7333
:101150000122B0FBF3F05146CBF80000584600F0F6
:10116000EFF918230293124B019380B240F255130A
:10117000CDE903A0009342464B46284600F068FDA7
:10118000237B2BB1FFF7C2FB237B002B7FF4F7AE51
:1011900013B0BDE8F08F00BF4C3300205D34002059
:1011A00000000240443300205834002078330020EF
:1011B0005C340020401DA12026812A0BF1C6A7C166
:1011C000D068080F903400204833002045330020B9
:1011D0003423002070B502F0D7F9094E094D308054
:1011E000002428683388834208D902F0C7F92B68A5
:1011F00004440133B4F5803F2B60F2D370BD00BFCF
:101200008C3400206034002002F082BA00F10060CB
:10121000920000F5803002F005BA0000054B1A6814
:10122000054B1B889B1A834202D9104402F0A6B9D1
:1012300000207047603400208C34002038B5084D01
:10124000044629B128682044BDE8384002F0B6B908
:101250002868204402F09AF90028F3D038BD00BF76
:1012600060340020064991F8243033B10023086A25
:1012700081F824300822FFF7C9BF0120704700BF62
:1012800064340020022802BF024B4FF080629A6152
:10129000704700BF00000240022802BF024B4FF41B
:1012A00080629A61704700BF0000024010B50023C1
:1012B000934203D0CC5CC4540133F9E710BD000065
:1012C00003460246D01A12F9011B0029FAD17047D1
:1012D00002440346934202D003F8011BFAE7704729
:1012E0002DE9F8431F4D144695F8242007468846FB
:1012F00052BBDFF870909CB395F824302BB92022B4
:10130000FF2148462F62FFF7E3FF95F82400C0F164
:101310000802A24228BF2246D6B24146920005EBFF
:101320008000FFF7C3FF95F82430A41B1E44F6B2DB
:10133000082E17449044E4B285F82460DBD1FFF70F
:1013400091FF0028D7D108E02B6A03EB8203834288
:10135000CFD0FFF787FF0028CBD10020BDE8F8836E
:101360000120FBE76434002000B59BB0EFF3098156
:1013700068226846FFF79AFFEFF30583044B9A6BE8
:10138000DA6A9A6A9A6A9A6A9A6A9A6A9B6AFEE71B
:1013900000ED00E000B59BB0EFF3098168226846DC
:1013A000FFF784FFEFF30583044B9A6B9A6A9A6AFE
:1013B0009A6A9A6A9A6A9B6AFEE700BF00ED00E0AB
:1013C00000B59BB0EFF3098168226846FFF76EFF16
:1013D000EFF30583034B5A6B9A6A9A6A9A6A9A6A80
:1013E0009B6AFEE700ED00E0FEE7000002F0CAB9EC
:1013F00002F0A2B92DE9F0470D46044600219046BF
:10140000284640F27912FFF763FF2346202200218D
:10141000284600F06DFE231D02222021284600F000
:1014200067FE631D03222221284600F061FEA31DF2
:1014300003222521284600F05BFE04F10803102258
:101440002821284600F054FE04F110030822382118
:10145000284600F04DFE04F11103082240212846E1
:1014600000F046FE04F1120308224821284600F04D
:101470003FFE04F1140320225021284600F038FEDC
:1014800004F1180340227021284600F031FE04F1D7
:1014900020030822B021284600F02AFE04F121038F
:1014A0000822B821284600F023FE04F12207C026B6
:1014B0003B46314608222846083600F019FEB6F5AC
:1014C000A07F07F10107F3D104F13203082231466E
:1014D000284600F00DFE002704F1330A94F832305C
:1014E0004FEAC7099F4209F5A47615D3B8F1000F5A
:1014F00008D1314604F599730722284600F0F8FD1B
:1015000009F24F16274694F832213B1B93420CD325
:10151000F01DC008BDE8F0870AEB0703082231463A
:10152000284600F0E5FD0137D8E707F233133146CE
:101530000822284600F0DCFD08360137E3E700000A
:1015400013B504460846002101602346C0F8031085
:101550002022019000F0CCFD0198231D02222021C1
:1015600000F0C6FD0198631D0322222100F0C0FD9A
:101570000198A31D0322252100F0BAFD019804F172
:1015800008031022282100F0B3FD072002B010BD8F
:10159000F8B50E4605461446002181223046FFF775
:1015A00097FE2B4608220021304600F0A1FD7CB9B1
:1015B0006B1C07220821304600F09AFD0F240123FE
:1015C0006A785F1C013B934204D3E01DC008F8BD5C
:1015D0000824F4E7EB1921460822304600F088FD84
:1015E00008343B46ECE7000030B5094D0A4491420F
:1015F0000DD011F8013B5840082340F30004013B93
:101600002C4013F0FF0384EA5000F6D1EFE730BD21
:101610002083B8EDF7B54FF0FF33DFF854C0DFF8A3
:1016200054E000EB81011A4688421CD050F8044B6C
:10163000019401AF042417F8015B82EA05620825D2
:10164000DB18164605F1FF355241002EBCBF83EA78
:101650000C0382EA0E0215F0FF05F1D1013C14F0F3
:10166000FF04E8D1E0E7D843D14303B0F0BD00BFA9
:101670009336EAA9EBE1F04273B5364A1068516837
:101680006B4603C36A4634493448082302F07EFCA3
:10169000044670B9324A106851686B4603C36A4603
:1016A00030492E48082302F071FC044620BB0A2072
:1016B00020E00369B3F5E02FECD8428B522AE9D140
:1016C000294A024402F110018B42E3D3103B234923
:1016D00000209D1AFFF788FF2A46064604F11801EC
:1016E0000020FFF781FFA3689E42D3D1E3689842B0
:1016F000D0D1002002B070BD0369B3F5E02F20D82F
:10170000B0F86620522A1ED1174A024402F15C0149
:101710008B421AD35C3B114900209D1AFFF764FFEE
:101720002A46064604F164010020FFF75DFFA26827
:10173000964203460BD1E068834214BF0D2000207F
:10174000D8E70B20D6E70C20D4E71020D2E70D20F5
:10175000D0E700BFFC3F0008DCFF060000000108E6
:101760000540000890FF06000800FFF72DE9F04152
:10177000C56915B9C161BDE8F0814B6823F06047C8
:10178000C3F38A464FEAD37EC3F3807816EA230672
:1017900038BF3E46AC462B465A68BEEBD27F22F09D
:1017A00060440AD0002A18DAA40CB44217D19D4232
:1017B0000FD10D60DEE71346EEE7A74207D102F036
:1017C0008044C2F3807242450BD054B1EFE708D297
:1017D000EDE7CCF800100B60CDE7B44201D0B44285
:1017E000E5D81A689C46002AE5D11960C3E70000D5
:1017F0002DE9F047089D01F007044FEAD50822447F
:1018000005F0070500EBD1004FF47F49944201D168
:10181000BDE8F08704F0070705F0070A57453E4684
:1018200038BF5646C6F10806111B8E4228BF0E4629
:10183000E10808EBD50E415C13F80EC0B94029FA57
:1018400006F721FA0AF1FFB28CEA010147FA0AF71A
:1018500039408CEA010C03F80EC034443544D5E716
:1018600080EA0120082341F2210201B24000002950
:1018700080B203F1FF33B8BF504013F0FF03F4D13F
:101880007047000038B50C468D18A54200D138BD10
:1018900014F8011BFFF7E4FFF7E7000002684AB104
:1018A00013680360C388018901339BB29942C380E6
:1018B00038BF03811046704770B588B020220446B7
:1018C0000D4668460021FFF703FD20460495FFF70B
:1018D000E5FF024658B16B46054608AE1C4603CCF0
:1018E000B44228606960234605F10805F6D1104628
:1018F00008B070BD082817D909280CD00A280CD0C8
:101900000B280CD00C280CD00D280CD00E2814BF9E
:101910004020302070470C20704710207047142062
:10192000704718207047202070470000082817D9FA
:101930000C280CD910280CD914280CD918280CD92B
:1019400020280CD930288CBF0F200E20704709208A
:1019500070470A2070470B2070470C2070470D20FD
:101960007047000010B54B6823B9CA8A63F30902B7
:10197000CA8210BDC4681A681C60C360438A013BF8
:1019800043824A60EFE700002DE9F84F1D46CB8AFD
:101990000F46C3F309010529814692460B4630D014
:1019A0000020AAB207F11A049EB2042E1FFA80F892
:1019B0000FD8904503F1010306D3FB8A0A4462F372
:1019C0000903FB8201201AE01AF80060E654013096
:1019D000EAE79045F1D2A1F1050B1C237C68BBFB23
:1019E000F3F203FB12BB1FFA8BF6002C45D14846DD
:1019F000FFF754FF044638B978606FF00200BDE885
:101A0000F88F4FF00008E6E7002606607860ADB278
:101A10004FF0000B454510D90AEB0803221D13F8BF
:101A2000011B9155B1B208F101081B291FFA88F872
:101A30002BD0454506F10106F1D8FB8AC3F3090214
:101A4000154465F30903BCE7013292B21C462368D2
:101A5000002BF9D16B1F0B441C21B3FBF1F30133B5
:101A60009BB29A42D3D2BBF1000FD0D14846FFF7C8
:101A700015FF20B9C4F800B0BFE70122E7E7C0F8BE
:101A800000B05E4620600446C1E74545D5D94846CA
:101A9000FFF704FF08B92060AFE7C0F800B00026E8
:101AA00020600446B6E700002DE9F04F2DED028BD3
:101AB00083B0CDE90013BDF83C5007469146002A9B
:101AC00000F092802DB10E9B002B00F08D80072D31
:101AD00032D807F10C00FFF7E1FE044638B96FF089
:101AE0000204204603B0BDEC028BBDE8F08F142247
:101AF0000021FFF7EDFB0E992A4604F10800FFF7DD
:101B0000D5FB681CC0B2FFF711FFFFF7F3FE20748E
:101B100099F80030013814FA80F003F01F0363F0E5
:101B20003F030372009B43F0004161603846214649
:101B3000FFF71CFE0124D4E700F10C034FF000086E
:101B400008EE103A4FF0800A4646444618EE100A56
:101B5000FFF7A4FE83460028C1D014220021FFF71E
:101B6000B7FBC6BB019BABF8083002200E9B00F10F
:101B7000080299195BFA82F20130C0B2082801D03C
:101B8000AE422AD3FFF7D2FEFFF7B4FE99F8002049
:101B9000009B411E02F01F0242EA4812AE4208BFFB
:101BA0004FF0400A5BFA81F14AEA020A43F0004230
:101BB00081F808A08BF81000CBF80420594638466D
:101BC000FFF7D4FD0134AE4224B288F001084FF093
:101BD000000ABBD185E70020C8E711F801CB02F865
:101BE00001CB0136B6B2C7E76FF0010479E7000018
:101BF000F8B515460E462822002104461F46FFF779
:101C000067FB069B6360B5F5001F079BA76034BFA9
:101C10006A094FF6FF72236204F10C0097B20023A9
:101C20009A4205D80023036027826382A382F8BD0D
:101C30000660013330462036F2E7000003781BB916
:101C40004BB2002BC8BF017070470000007870478E
:101C50002DE9F74FDDF83C90BDF830500D9E9DF812
:101C60003840BDF84070804692469B46B9F1000F5F
:101C700001D1002F51D11F2C4FD898F80000B0B9D6
:101C8000072F47D835F0030347D13A4649464FF668
:101C9000FF70FFF7F7FD20F001002D02400445EA38
:101CA0000464400C44EA40244FF6FF7321E040EA0C
:101CB0000520072F40EA0464F6D900254FF6FF738C
:101CC000C5F12000A5F120022AFA05F10BFA00F077
:101CD00001432BFA02F211431846C9B2FFF7C0FDC7
:101CE0000835402D0346EBD13A464946FFF7CAFD79
:101CF0000346CDE90097324621464046FFF7D4FE21
:101D000033780133DBB21F2B88BF0023337003B05D
:101D1000BDE8F08F6FF00300F9E76FF00100F6E720
:101D20002DE9F04F85B09246DDF848800F9D9DF873
:101D300040209DF84490BDF84C7006469B46B8F193
:101D4000000F01D1002F48D11F2A46D83378002B2D
:101D500046D00C0244EA02649DF8381044EAC934C3
:101D600044EA01441C43072F44F0800432D9002385
:101D70004FF6FF72C3F1200CA3F120002AFA03F101
:101D80000BFA0CFC41EA0C012BFA00F00143C9B23A
:101D900010460393FFF764FD039B0833402B024674
:101DA000E8D13A464146FFF76DFD0346CDE900878D
:101DB0002A4621463046FFF777FEB9F1010F06D1DA
:101DC0002B780133DBB21F2B88BF00232B7005B0AB
:101DD000BDE8F08F4FF6FF73E8E76FF00100F6E71C
:101DE0006FF00300F3E70000C06900B104307047F2
:101DF000C3691A68C261C2681A60C360438A013B42
:101E0000438270472DE9F041D0F81880194E1446EE
:101E10001D464146002709B9BDE8F081D1E90223FA
:101E2000A21A65EB0303964277EB03031ED2836984
:101E30008B420DD1FFF796FD83691B688361C368F0
:101E40000B60438AC1608169013B43828846E2E7B7
:101E5000FFF788FD0B68C8F80030C3680B60438A41
:101E6000C160013B4382D8F80010D4E78846096876
:101E7000D1E700BF80841E002DE9F04F8BB00D46E6
:101E8000DDF8509014469B468046002800F01981EA
:101E9000B9F1000F00F01581531E3F2B00F21181A4
:101EA000012A03D1BBF1000F40F00B810023CDE9E3
:101EB0000833B8F81430B5EBC30F4FEAC30703D3A8
:101EC00000200BB0BDE8F08F2B199F42D8F80C30E2
:101ED0003ABF7F1BFFB227461BB9D8F81030002B42
:101EE0007AD0272D4ED8C5F12806B7424FF000030F
:101EF0002CBFF6B23E4600932946D8F8080008AB3E
:101F00003246FFF775FCA7EB060A35445FFA8AFAFA
:101F1000B8F8143003F10053053BDB000493D8F804
:101F20000C3003932821039B13B1BAF1000F2CD17D
:101F3000D8F8100040B1BAF1000F05D0009608ABF8
:101F40005246691AFFF754FC38B2002FB8D0660722
:101F50000AD00AAB03EBD401624211F8083C02F04C
:101F60000702134101F8083C082C3CD9102C40F220
:101F7000B580202C40F2B780BBF1000F00F09C80B0
:101F8000082334E0BA460026C2E7049BE02B28BFB2
:101F9000E02306930B44AB42059314D95A1B0398D4
:101FA0000096924534BF5246D2B2691A08AB04304B
:101FB0000792FFF71DFC079A1644AAEB020A154484
:101FC000F6B25FFA8AFA049B069A05999B1A049363
:101FD000039B1B680393A6E70093D8F8080008AB9F
:101FE0003A462946AEE7BBF1000F13D00123B4EB0C
:101FF000C30F6CD0082C12D89DF82030621E23FA33
:1020000002F2D50706D54FF0FF3202FA04F423435B
:102010008DF820309DF8203089F8003051E7102CE1
:1020200012D8BDF82030621E23FA02F2D10706D57D
:102030004FF0FF3202FA04F42343ADF82030BDF82C
:102040002030A9F800303CE7202C0FD80899631EF7
:1020500021FA03F3DA0705D54FF0FF3202FA04F450
:102060000C430894089BC9F800302AE7402C2BD079
:10207000DDE90865611EC4F12102A4F1210326FAFD
:1020800001F105FA02F225FA03F311431943CB07D4
:1020900012D50122A4F12003C4F1200102FA03F3B6
:1020A00022FA01F1A240524243EA010363EB4303E7
:1020B00032432B43CDE90823DDE90823C9E9002396
:1020C000FFE66FF00100FCE66FF00800F9E6082C6F
:1020D000A0D9102CB3D9202CEED8C3E7BBF1000F48
:1020E000ADD0022383E7BBF1000FBBD004237EE712
:1020F00030B5012A144638BF0124402C85B028BFD2
:1021000040240025012ACDE9025518D81B788DF806
:10211000083063070AD004AB03EBD405624215F81C
:10212000083C02F00702934005F8083C0091034682
:102130002246002102A8FFF75BFB05B030BD082A4C
:10214000E4D9102A03D81B88ADF80830E1E7202A2B
:102150008DBFD3E900231B680293CDE90223D8E7A2
:1021600010B5CB681BB98B600B618B8210BDC46846
:102170001A681C60C360438A013B4382CA60F0E76F
:102180002DE9F04F95B0CDE904230B6804460D46C8
:102190001806C3F3C01147BFC3F3C03BC3F3062601
:1021A0004FF0020B0E46002B80F2018213F0C04963
:1021B00040F0FD812A7B002A00F0F981BBF1020F7B
:1021C00003D02078B04240F0F581C3F3046008905A
:1021D00003F07F00069069B3C3F3074A2A44069BC5
:1021E00092F80380760646EA0B4646EA83460022CA
:1021F0000023CDE90A235FEAD81346EA0A060393CF
:102200006CD0069B009367685B4652460AA920463D
:10221000B847002800F0D181A76997B9314604F189
:102220000C00FFF749FB0746D8B96FF0020015B064
:10223000BDE8F08FC3F30F2A590608BF0AF0030A5E
:10224000CCE73B699E420DD03F68002FF9D1314663
:1022500004F10C00FFF730FB07460028E5D0A36926
:102260003B60A761FE7D08F01F03C6F38406F01AE9
:102270001FFA80FC0028B8BF0CF120000793A3EBE5
:1022800006031FFA83FCD7E90221B8BF00B2002B76
:102290000993BEBF0CF120031BB2099352EA01035C
:1022A00033D0049EDFF8D0C2B21A059E66EB01015E
:1022B0000026944576EB010327D395F80DE097F8B7
:1022C0001AC0E64514D1039B002B76D001281CDCF4
:1022D000A848904276EB010314D336E0A76917B9FA
:1022E0006FF00C00A3E73B699E42BBD03F68F6E766
:1022F000A048904276EB010301D3002097E7039BAF
:10230000002BFAD0099B0F2B18DCFA7D4FEA8803CB
:1023100002F0030203F07C031343FB7539462046A9
:10232000FFF720FB6B7BBB76039B3BB9FB7DC3F3C5
:102330008402013262F38603FB75D1E76A7BBB7EC0
:102340009A42DAD1039B002B37D04FEA9813022B25
:1023500033D0049BBB60059BFB60142200210FA8B7
:10236000FEF7B6FF049B0C93059B0D932B1D0E935C
:102370002B7BADF846A0013BDBB2ADF84430079BA8
:102380008DF84930089B8DF84A30069B8DF84B300C
:1023900094F824308DF848B083F001038DF84C3068
:1023A0000CA9A36820469847FB7DC3F3840301333F
:1023B00003F01F039B02FB829FE7FB7DC8F34012E3
:1023C000B2EBD31F40F0FC80079AC3F3840393421F
:1023D00040F0F98003992B7B4FEA981200294ED0E8
:1023E000D2075ED4032B40F2F180049BBB60059BB7
:1023F000FB602B7BAE1D033BDBB23246394604F15A
:102400000C00FFF7C1FA00280DDA20463946FFF725
:10241000A9FAFB7DC3F38403013303F01F039B027E
:10242000FB82032003E7DDE90A84AB883B834FF698
:10243000FF73C9F12000A9F1200228FA09F104FA7A
:1024400000F0014324FA02F211431846C9B2FFF723
:1024500007FA09F10809B9F1400F0346E9D1B8823A
:102460002A7B033AD2B23146FFF70CFAFB7DB882E1
:10247000DA43C2F3C01262F3C713FB753DE782B9BA
:102480002E1D013BDBB23246394604F10C00FFF74A
:102490007BFA0028B9DB2A7BB88A013AD2B23146EE
:1024A000E2E7F98AC1F30901013B0429DAB25BD8FA
:1024B000281D002307F11B069A4208D910F801CB0A
:1024C00006F801C0013101330529DBB2F4D10499CA
:1024D0000C9105990D91934207F11B010E9138BFA4
:1024E000043379680F9134BF55FA83F300231093B6
:1024F000FB8AADF846A0C3F309031A44079B8DF885
:102500004930089B8DF84A30069B8DF84B3094F883
:102510002430ADF8442083F001038DF84C300023C3
:102520008DF848B07B602A7BB88A013A291DFFF7F5
:10253000A9F93B8BB882834203D1A3680CA920463A
:10254000984720460CA9FFF70BFEFB7DB88AC3F322
:102550008403013303F01F039B02FB823B8B9842F1
:1025600014BF1120002062E67B68002BAFD005204D
:1025700006E000BF40420F0080841E001C3033463E
:102580001E68002EFAD1091A081D2E1D184401EBF1
:10259000090CBCF11B0F5FFA89F398D89A4296D9BF
:1025A00016F8013B00F8013B09F10109EFE76FF074
:1025B00009003CE66FF00A0039E66FF00B0036E6E2
:1025C0006FF00D0033E66FF00E0030E66FF00F0095
:1025D0002DE600BF404BF0B51C6C404E44F000743B
:1025E0001C641D6E45F000751D661B6E3C4B9B6A9E
:1025F000D3F80052354045F00105C3F80052D3F836
:102600000042344044EA002040F00100C3F80002D8
:10261000002952D00020C3F81C020546C3F804026A
:10262000C3F80C02C3F8140203EBC00401301C28E9
:10263000C4F84052C4F84452F6D100254FF0010CC2
:1026400096781488F70748BFD3F804720CFA04F0A0
:1026500044BF0743C3F80472B70742BFD3F80C72F4
:102660000743C3F80C72760742BFD3F814620643DF
:10267000C3F8146203EBC4045668C4F84062966859
:10268000C4F84462D3F81C4201352043A942C3F880
:102690001C0202F10C02D3D1D3F8002222F0010275
:1026A000C3F800220C4B1A6C22F000721A641A6EE6
:1026B00022F000721A661B6EF0BD0122C3F84012B0
:1026C000C3F84412C3F80412C3F81412C3F80C225E
:1026D000C3F81C22E0E700BF003802400000FFFF03
:1026E00090340020184A916A08B58B688B6013F00B
:1026F000010104D013F00C0F18BF4FF48031D8053E
:1027000006D513F4406F14BF41F4003141F00201CB
:10271000D80306D513F4402F14BF41F4802141F0B3
:102720000401D3690BB108489847202383F311882B
:102730000648002100F0EEFD002383F31188BDE878
:10274000084001F017B900BF9034002098340020F1
:1027500038B5124CA36ADD68AA0712D05A6922F074
:1027600002025A61A36913B1012120469847202330
:1027700083F311880A48002100F0CCFD002383F385
:102780001188EB0606D5A36A1021D960236A0BB124
:1027900002489847BDE8384001F0ECB8903400207A
:1027A000A034002038B5124CA36A1D69AA0712D0C4
:1027B0005A6922F010025A61A36913B1022120461E
:1027C0009847202383F311880A48002100F0A2FDD6
:1027D000002383F31188EB0606D5A36A1021196143
:1027E000236A0BB102489847BDE8384001F0C2B8EF
:1027F00090340020A034002038B50F4CA36A5D68E7
:102800005D602A070AD5042222701A6822F00202AB
:102810001A60636A13B10021204698476B0706D5FA
:10282000A36A9969236A13B1034809049847BDE86C
:10283000384001F09FB800BF9034002010B50E4C16
:10284000204600F0CFF90D4BA3620B21132000F0BE
:10285000B1F90B21142000F0ADF90B21152000F087
:10286000A9F90B21162000F0A5F90022BDE81040BF
:1028700011460E20FFF7AEBE9034002000640040E9
:10288000114B984210B5044609D1104B1A6C42F016
:1028900000721A641A6E42F000721A661B6EA36A06
:1028A00001221A60A36A5A68D20707D56268516884
:1028B0001268D9611A60064A5A6110BD01210820C8
:1028C00000F01EFCEEE700BF90340020003802400C
:1028D0005B87010003291AD8DFE801F0020A0F1410
:1028E000836A9B6813F0E05F14BF012000207047EB
:1028F000836A9868C0F380607047836A9868C0F301
:10290000C0607047836A9868C0F300707047002009
:102910007047000010B5032925D8DFE801F0022533
:10292000292D836A9968C1F30161183103EB011302
:10293000107884064CBF54689488C0F300114FEAA5
:10294000410148BF41EAC40100F00F004CBF41F013
:10295000040141EA4451586041F001019068D26895
:102960009860DA60196010BD836A03F5C073DFE711
:10297000836A03F5C873DBE7836A03F5D073D7E78F
:1029800001290AD002290FD081B9836ADA68920737
:1029900001D1186903E001207047836AD86810F0FC
:1029A000030018BF01207047836AF2E700207047D8
:1029B00010B539B9836AD96889071BD11B699C078F
:1029C00004D110BD012915D00229FAD1816AD1F8AC
:1029D000C031D1F8C441D1F8C8011061D1F8CC019F
:1029E0005061202008610869800717D1486940F0CC
:1029F000100012E0816AD1F8B031D1F8B441D1F8B9
:102A0000B8011061D1F8BC0150612020C860C868CD
:102A1000800703D1486940F002004861C3F34000D9
:102A2000C3F38001000140EA4111107920F0300029
:102A30000143117189064BBF91681189DB085B0D59
:102A40004CBF63F31C0163F30A01137948BF916023
:102A500064F3030313714FEA14234FEA144458BF7D
:102A6000118113705480ACE7024AD36843F0C0036D
:102A7000D360704700440040044B5A6810439A6882
:102A800058600AB1181D1047704700BFBC340020C1
:102A90002DE9F0413C4ED6F85C52EF682B68DA0520
:102AA0009CB20CD5202383F311884FF40070FFF7FC
:102AB000E3FF6FF480732B60002383F311882023DE
:102AC00083F31188DFF8C08014F02F0339D183F32A
:102AD0001188380613D5210611D5202383F31188D8
:102AE0002A4800F001FA00284CDA0820FFF7C4FF5A
:102AF0004FF67F733B40EB60002383F311887A0627
:102B000015D5630613D5202383F31188D6E9132343
:102B10009A4209D1336C3BB127F040073F041020A3
:102B20003F0CFFF7A9FFEF60002383F31188D6F86D
:102B30006422D3680BB110699847BDE8F04100F0FA
:102B400019BF230712D014F0080F0CBF00208020FB
:102B5000E10748BF40F02000A20748BF40F0400016
:102B6000630748BF40F48070FFF786FFA4066B68D8
:102B700005D596F860124046194000F057FA2C68C7
:102B8000A4B2A1E76860B7E7BC340020F4340020A9
:102B900010B5054C054A0021204600F025FA044BEB
:102BA000C4F85C3210BD00BFBC340020692A0008A4
:102BB0000044004000F1604303F561430901C9B2DC
:102BC00083F80013012200F01F039A4043099B0081
:102BD00003F1604303F56143C3F880211A60704735
:102BE000FFF72CBE012300F10802C0E902220370A6
:102BF00000F110020023C0E90422C0E90633C0E955
:102C0000083343607047000010B52023044683F367
:102C10001188022303704160FFF732FE0423237002
:102C2000002383F3118810BD2DE9F0411F460446AF
:102C30000D461646202383F3118800F108082378F7
:102C4000052B0DD029462046FFF744FE40B1204613
:102C500032462946FFF75EFE002080F3118808E027
:102C60003946404600F03AFB0028E8D0002383F3C1
:102C70001188BDE8F08100002DE9F0411F460446AF
:102C80000D461646202383F3118800F1100823789F
:102C9000052B0DD029462046FFF772FE40B1204695
:102CA00032462946FFF784FE002080F3118808E0B1
:102CB0003946404600F012FB0028E8D0002383F399
:102CC0001188BDE8F0810000F8B5154682680669F4
:102CD000AA420B46816938BF8568761AB542044618
:102CE0000BD218462A46FEF7E1FAA3692B44A361EA
:102CF000A3685B1BA3602846F8BD0CD91846324672
:102D0000FEF7D4FAAF1BE1683A463044FEF7CEFA3C
:102D1000E3683B44EBE718462A46FEF7C7FAE36848
:102D2000E5E7000083689342F7B51546044638BFCF
:102D30008568D0E90460361AB5420BD22A46FEF700
:102D4000B5FA63692B446361A36828465B1BA360E3
:102D500003B0F0BD0DD932460191FEF7A7FA0199F3
:102D6000E068AF1B3A463144FEF7A0FAE3683B4403
:102D7000E9E72A46FEF79AFAE368E4E710B50A4461
:102D80000024C361029B8460C0E90000C0E9051112
:102D9000C1600261036210BD08B5D0E905329342FB
:102DA00001D1826882B98268013282605A1C426114
:102DB0001970D0E904329A4224BFC36843610021EC
:102DC00000F09CFA002008BD4FF0FF30FBE7000048
:102DD00070B5202304460E4683F31188A568A5B17B
:102DE000A368A269013BA360531CA3611578226903
:102DF000934224BFE368A361E3690BB1204698477F
:102E0000002383F31188284607E03146204600F06E
:102E100065FA0028E2DA85F3118870BD2DE9F74FD5
:102E200004460E4617469846D0F81C904FF0200AEC
:102E30008AF311884FF0000B154665B12A463146DA
:102E40002046FFF741FF034660B94146204600F0A7
:102E500045FA0028F1D0002383F31188781B03B0D2
:102E6000BDE8F08FB9F1000F03D001902046C847AC
:102E7000019B8BF31188ED1A1E448AF31188DCE75D
:102E8000C0E90511C160C3611144009B8260C0E9C3
:102E90000000016103627047F8B504460D4616460E
:102EA000202383F31188A768A7B1A368013BA3601F
:102EB00063695A1C62611D70D4E904329A4224BFCE
:102EC000E3686361E3690BB120469847002080F313
:102ED000118807E03146204600F000FA0028E2DAC7
:102EE00087F31188F8BD0000D0E905239A4210B598
:102EF00001D182687AB98268013282605A1C82618B
:102F00001C7803699A4224BFC3688361002100F0E2
:102F1000F5F9204610BD4FF0FF30FBE72DE9F74FE4
:102F200004460E4617469846D0F81C904FF0200AEB
:102F30008AF311884FF0000B154665B12A463146D9
:102F40002046FFF7EFFE034660B94146204600F0F9
:102F5000C5F90028F1D0002383F31188781B03B052
:102F6000BDE8F08FB9F1000F03D001902046C847AB
:102F7000019B8BF31188ED1A1E448AF31188DCE75C
:102F8000026843681143016003B1184770470000AD
:102F90001430FFF743BF00004FF0FF331430FFF74A
:102FA0003DBF00003830FFF7B9BF00004FF0FF33DE
:102FB0003830FFF7B3BF00001430FFF709BF00003F
:102FC0004FF0FF311430FFF703BF00003830FFF738
:102FD00063BF00004FF0FF323830FFF75DBF0000E5
:102FE00000207047FFF7D4BD37B515460E4A026082
:102FF00000224260C0E902220122044602740B460C
:10300000009000F15C014FF480721430FFF7B6FEBF
:1030100000942B464FF4807204F5AE7104F1380031
:10302000FFF72EFF03B030BD1040000838B5C3696C
:1030300004460D461BB904210844FFF7A1FF2946A9
:1030400004F11400FFF7A8FE002806DA201D4FF453
:103050008061BDE83840FFF793BF38BD024B0022C6
:10306000C3E900339A6070472437002000230374BB
:103070008268054B1B6899689142FBD25A680360CD
:1030800042601060586070472437002008B5202344
:1030900083F31188037C032B05D0042B0DD02BB9AF
:1030A00083F3118808BD436900221A604FF0FF3393
:1030B0004361FFF7DBFF0023F2E7D0E90032136042
:1030C0005A60F3E7002303748268054B1B68996814
:1030D0009142FBD85A6803604260106058607047A4
:1030E00024370020054B19690874186802681A60B3
:1030F0005360186101230374FDF78ABA2437002056
:1031000030B54B1C0B4D87B0044610D02B690A4AD2
:1031100001A800F01BF92046FFF7E4FF049B13B160
:1031200001A800F04FF92B69586907B030BDFFF7CF
:10313000D9FFF8E7243700208D30000838B50C4D52
:1031400041612B6981689A689142044603D8BDE8C1
:103150003840FFF78BBF1846FFF7B4FF01232C61FF
:10316000014623742046BDE83840FDF751BA00BF40
:1031700024370020044B1A681B6990689B689842AA
:1031800094BF0020012070472437002010B5084C60
:10319000236820691A6822605460012223611A742E
:1031A000FFF790FF01462069BDE81040FDF730BAF7
:1031B0002437002008B5FFF7DDFF18B1BDE808404F
:1031C000FFF7E4BF08BD0000FFF7E0BFFEE7000027
:1031D00010B50C4CFFF742FF00F0AAF80A49802214
:1031E000204600F031F8012344F8180C037400F075
:1031F0009DFB002383F3118862B60448BDE81040AC
:1032000000F042B84C370020384000084840000821
:1032100000F012B9EFF3118020B9EFF305832022FB
:1032200082F311887047000010B530B9EFF30584C0
:10323000C4F3080414B180F3118810BDFFF7BAFF7E
:1032400084F31188F9E7000082600222028270474D
:103250008368A3F17C0243F80C2C026943F83C2CF0
:10326000426943F8382C074A43F81C2CC26843F8DB
:10327000102C022203F8082C002203F8072CA3F1DB
:10328000180070472906000810B5202383F3118821
:10329000FFF7DEFF00210446FFF750FF002383F312
:1032A0001188204610BD0000024B1B6958610F2099
:1032B000FFF718BF24370020202383F31188FFF77E
:1032C000F3BF000008B50146202383F311880820CE
:1032D000FFF716FF002383F3118808BD49B1064BA1
:1032E00042681B6918605A60136043600420FFF74E
:1032F00007BF4FF0FF307047243700200368984223
:1033000006D01A680260506059611846FFF7AEBED9
:103310007047000038B504460D462068844200D14D
:1033200038BD036823605C604561FFF79FFEF4E7EA
:10333000054B03F11402C3E905224FF0FF310022CF
:10334000C3E90712704700BF2437002070B51C4E38
:10335000C0E9032305460C4600F06EFB334653F8E4
:10336000142F9A420DD13062C5E901242A600A2C3B
:103370002CBF00190A30C6E90555BDE8704000F0C1
:1033800049BB316A431AE31838BF1C469368A3420D
:1033900002D9081900F04CFB73699A6894420CD862
:1033A0005A68AC602B606A6015609A685D60121B99
:1033B0009A604FF0FF33F36170BD1B68A41AECE70D
:1033C0002437002038B51B4C636998420DD0D0E9F2
:1033D000003213605A6000228168C2609A680A4411
:1033E0009A604FF0FF33E36138BD2246036842F82C
:1033F000143F002193425A60C16003D1BDE83840B8
:1034000000F010BB9A688168256A0A449A6000F04F
:1034100013FB63699A68411B8A42E5D9AB181D1AF0
:10342000092D206A98BF01F10A02BDE83840104416
:1034300000F0FEBA243700202DE9F041184C002797
:1034400004F11406656900F0F7FA236AAA68C11A44
:103450008A4215D813442362D5E9003213605A60BA
:103460006369D5F80C80EF60B34201D100F0DAFA5D
:1034700087F311882869C047202383F31188E1E787
:103480006169B14209D013441B1ABDE8F0410A2B0F
:103490002CBFC0180A3000F0CBBABDE8F08100BFE5
:1034A0002437002000207047FEE70000704700002E
:1034B0004FF0FF3070470000BFF34F8F024AD368D0
:1034C000DB03FCD4704700BF003C024008B5094B49
:1034D0001B7873B9FFF7F0FF074B1A69002ABFBFCB
:1034E000064A5A6002F188325A601A6822F48062F1
:1034F0001A6008BDE0380020003C02402301674507
:1035000008B50B4B1B7893B9FFF7D6FF094B1A6927
:1035100042F000421A611A6842F480521A601A6836
:1035200022F480521A601A6842F480621A6008BD60
:10353000E0380020003C02400728F0B516D80C4CBB
:103540000C4923787BB90C4D0E4608234FF00062DE
:1035500055F8047B46F8042B013B13F0FF033A4473
:10356000F6D10123237051F82000F0BD0020FCE7C4
:1035700004390020E438002060400008014B53F873
:10358000200070476040000808207047072810B5E9
:10359000044601D9002010BDFFF7CEFF064B53F8BB
:1035A00024301844C21A0BB90120F4E71268013222
:1035B000F0D1043BF6E700BF60400008072838B5AB
:1035C000044628D8FFF726FEFFF776FFFFF77EFFB9
:1035D000124AF323D360E300DBB243F4007343F0F9
:1035E00002031361136943F48033136105462046D7
:1035F000FFF762FFFFF7A0FF094B53F8241000F01C
:103600003BF92846FFF77CFFFFF70EFE2046BDE89A
:103610003840FFF7BBBF002038BD00BF003C024070
:103620006040000812F001032DE9F04105460E4606
:1036300014464BD18118334A914261D8324B1B68F2
:1036400013F001035CD0314FFFF7E4FDFFF73EFFBD
:10365000F323FB60FFF730FF314640F20128032CD3
:1036600018D824F00104294E0C446D1A40F20118B8
:10367000A142336905EB01072AD123F0010333612D
:10368000FFF73EFFFFF7D0FD0120BDE8F081043CCD
:103690000435E4E7AB07E4D13B6923F440733B61B5
:1036A0003B6943EA08033B6151F8046B2E60BFF3AA
:1036B0004F8FFFF701FF2B689E42E8D03B6923F054
:1036C00001033B61FFF71CFFFFF7AEFD0020DCE7C5
:1036D00023F440733361336943EA080333610B8891
:1036E0003B80BFF34F8FFFF7E7FE3F8831F8023B87
:1036F000BFB2BB42BCD0336923F001033361E1E7C1
:103700001846C2E70000080800380240003C0240AA
:10371000084908B50B7828B11BB9FFF7D7FE01237C
:103720000B7008BD002BFCD0BDE808400870FFF707
:10373000E7BE00BFE038002070B582B0FFF76AFD39
:103740000E4E054600F078F93268904237BF0C4AB9
:103750000B49516814682EBFD1E900410131516015
:103760000419034641F10001284601913360FFF737
:103770005BFD0199204602B070BD00BF08390020F2
:103780001039002070B582B0FFF744FD104E054699
:1037900000F052F93268904237BF0E4A0D49516825
:1037A00014682EBFD1E9004101315160041941F183
:1037B00000010346284601913360FFF735FD01996A
:1037C0004FF47A7200232046FCF70AFD02B070BD68
:1037D000083900201039002010B50244064BD2B23F
:1037E000904200D110BD441C00B253F8200041F8B3
:1037F000040BE0B2F4E700BF502800400F4B30B597
:103800001C6F240407D41C6F44F400741C671C6FE5
:1038100044F400441C670A4C236843F4807323601B
:103820000244084BD2B2904200D130BD441C00B2D9
:1038300051F8045B43F82050E0B2F4E7003802404E
:10384000007000405028004007B5012201A9002067
:10385000FFF7C2FF019803B05DF804FB13B50446FF
:10386000FFF7F2FFA04205D0012201A90020019438
:10387000FFF7C4FF02B010BD70470000074B45F2D0
:1038800055521A6002225A6040F6FF729A604CF656
:10389000CC421A60024B01221A707047003000407F
:1038A0001C390020034B1B781BB1034B4AF6AA229C
:1038B0001A6070471C39002000300040034B1A6822
:1038C0001AB9034AD2F874281A60704718390020D0
:1038D00000300240024B4FF08072C3F874287047EA
:1038E0000030024008B5FFF7E9FF024B1868C0F34B
:1038F000407008BD1839002008B5FFF7DFFF024B04
:103900001868C0F3007008BD18390020EFF3098370
:1039100005494A6B22F001024A63683383F3098840
:10392000002383F31188704700EF00E0202080F32C
:10393000118862B60C4B0D4AD96821F4E061090484
:10394000090C0A43DA60D3F8FC20094942F080727E
:10395000C3F8FC200A6842F001020A601022DA77FC
:1039600083F82200704700BF00ED00E00003FA0575
:10397000001000E010B5202383F311880E4B5B6824
:1039800013F4006314D0F1EE103AEFF30984683CAD
:103990004FF08073E361094BDB6B236684F3098886
:1039A000FFF7E8FB10B1064BA36110BD054BFBE729
:1039B00083F31188F9E700BF00ED00E000EF00E0BD
:1039C0003B0600083E06000870470000FEE70000C6
:1039D0000A4B0B480B4A90420BD30B4BDA1C121AC2
:1039E000C11E22F003028B4238BF00220021FDF7E6
:1039F0006FBC53F8041B40F8041BECE78C41000833
:103A0000A0390020A0390020A03900207047000014
:103A100000F080B84FF08043002258631A61022200
:103A2000DA6070474FF080430022DA607047000090
:103A30004FF08043586370474FF08043586A704797
:103A40004B6843608B688360CB68C3600B694361DC
:103A50004B6903628B6943620B6803607047000027
:103A600008B5234B23481A6942F0FF021A611A690C
:103A700022F0FF021A611A691A6B42F0FF021A6300
:103A80001A6D42F0FF021A651B4A1B6D1146FFF7C3
:103A9000D7FF02F11C0100F58060FFF7D1FF02F1B2
:103AA000380100F58060FFF7CBFF02F1540100F50B
:103AB0008060FFF7C5FF02F1700100F58060FFF73D
:103AC000BFFF02F18C0100F58060FFF7B9FF02F142
:103AD000A80100F58060FFF7B3FF02F1C40100F513
:103AE0008060FFF7ADFFBDE8084000F097B800BF69
:103AF00000380240000002408040000808B500F095
:103B000017FAFFF765FBBDE80840FFF7D7BE0000D6
:103B100070470000104B1A6C42F001021A641A6ED2
:103B200042F001021A660D4A1B6E936843F00103CE
:103B300093604FF0804331229A624FF0FF32DA6295
:103B400000229A615A63DA605A6001225A610821A0
:103B50001A601C20FFF72EB800380240002004E055
:103B60004FF0804208B51169D3680B40D9B2C94300
:103B70009B07116107D5202383F31188FFF748FBCA
:103B8000002383F3118808BD08B5FFF7E9FFBDE8FE
:103B90000840FFF7EFBE00001E4B1A6962F0FF02FB
:103BA0001A611A69D2B21A614FF0FF301A695A6964
:103BB000586100215A6959615A691A6A62F0805243
:103BC0001A621A6A02F080521A621A6A5A6A5862B3
:103BD0005A6A59625A6A1A6C42F080521A641A6E12
:103BE00042F080521A661A6E0B4A106840F48070D8
:103BF0001060186F00F44070B0F5007F1EBF4FF4E6
:103C0000803018671967536823F40073536000F01D
:103C10006FB900BF00380240007000403B4B3C4A87
:103C20001A643C4A4FF4404111601A6842F00102A4
:103C30001A601A689007FCD59A6822F003029A600D
:103C4000324B9A6812F00C02FBD1196801F0F901AD
:103C500019609A601A6842F480321A601A689103F7
:103C6000FCD55A6F42F001025A67284B5A6F9207EF
:103C7000FCD5294A5A601A6842F080721A60254AB7
:103C800053685804FCD5214B1A689101FCD5234A8E
:103C9000C3F884201A6842F080621A601A68120120
:103CA000FCD51F4A9A600322C3F88C204FF00062B3
:103CB000C3F894201B4B1A681B4B9A421B4B21D113
:103CC0001B4A11681B4A91421CD140F203121A6030
:103CD000164A136803F00F03032BFAD10B4B9A68B3
:103CE00042F002029A609A6802F00C02082AFAD1A5
:103CF0005A6C42F480425A645A6E42F480425A66C8
:103D00005B6E704740F20372E1E700BF003802408B
:103D10000004001000700040041940020830002424
:103D200000948838002004E011640020003C024028
:103D300000ED00E041C20F41084A08B5516913681F
:103D40000B4003F00103536123B1054A13680BB123
:103D500050689847BDE80840FFF70CBE003C0140A2
:103D600020390020084A08B5516913680B4003F058
:103D70000203536123B1054A93680BB1D068984799
:103D8000BDE80840FFF7F6BD003C014020390020A7
:103D9000084A08B5516913680B4003F004035361E6
:103DA00023B1054A13690BB150699847BDE8084033
:103DB000FFF7E0BD003C014020390020084A08B56B
:103DC000516913680B4003F00803536123B1054A9E
:103DD00093690BB1D0699847BDE80840FFF7CABDA9
:103DE000003C014020390020084A08B55169136899
:103DF0000B4003F01003536123B1054A136A0BB162
:103E0000506A9847BDE80840FFF7B4BD003C014048
:103E100020390020174B10B55A691C68144004F46F
:103E200078725A61A30604D5134A936A0BB1D06A1B
:103E30009847600604D5104A136B0BB1506B984736
:103E4000210604D50C4A936B0BB1D06B9847E20561
:103E500004D5094A136C0BB1506C9847A30504D5DF
:103E6000054A936C0BB1D06C9847BDE81040FFF742
:103E700081BD00BF003C0140203900201A4B10B525
:103E80005A691C68144004F47C425A61620504D5E6
:103E9000164A136D0BB1506D9847230504D5134A8C
:103EA000936D0BB1D06D9847E00404D50F4A136EA3
:103EB0000BB1506E9847A10404D50C4A936E0BB118
:103EC000D06E9847620404D5084A136F0BB1506F47
:103ED0009847230404D5054A936F0BB1D06F9847D8
:103EE000BDE81040FFF746BD003C014020390020EE
:103EF000062108B50846FEF75DFE06210720FEF7FD
:103F000059FE06210820FEF755FE06210920FEF77E
:103F100051FE06210A20FEF74DFE06211720FEF76E
:103F200049FEBDE8084006212820FEF743BE0000F8
:103F300008B5FFF731FE00F00BF8FEF751FEFFF772
:103F400051F8FFF7E5FDBDE80840FFF761BD00004F
:103F50000023054A19460133102BC2E9001102F172
:103F60000802F8D1704700BF2039002010B5013990
:103F70000244904201D1002005E0037811F8014F7E
:103F8000A34201D0181B10BD0130F2E72DE9F0412A
:103F9000A3B1C91A17780144044603F1FF3C8C42CF
:103FA000204601D9002009E00578BD4204F1010452
:103FB000F5D10CEB0405D618A54201D1BDE8F0817E
:103FC00015F8018D16F801EDF045F5D0E7E7000092
:103FD000034611F8012B03F8012B002AF9D1704791
:103FE0006F72672E6172647570696C6F742E4152C6
:103FF0004B5F52544B5F47505300000040A2E4F126
:10400000646891060041A3E5F2656992070000002B
:1040100000000000AD2F0008992F0008D52F0008E0
:10402000C12F0008CD2F0008B92F0008A52F0008C8
:10403000912F0008E12F00086D61696E00000000FB
:1040400069646C650000000040400008683700208B
:10405000E038002001000000CD3100080000000021
:104060000040000000400000004000000040000050
:104070000000010000000200000002000000020039
:10408000A000902A00000000AAAAAAAA50000024BA
:10409000FFFB000000770000009009000100000510
:1040A00000000000AAAAAAA501000080FFEF0000FE
:1040B0000000000000000000000000000000000000
:1040C000AAAAAAAA00000000FFFF0000000000004A
:1040D000000000000000000000000000AAAAAAAA38
:1040E00000000000FFFF00000000000000000000D2
:1040F0000000000000000000AAAAAAAA0000000018
:10410000FFFF0000000000000000000000000000B1
:1041100000000000AAAAAAAA00000000FFFF0000F9
:10412000000000000000000000000000000000008F
:10413000AAAAAAAA00000000FFFF000000000000D9
:104140000000000000000000000000000A00000065
:10415000000000000300000000000000000000005C
:10416000B0C0FF7F0100000052000000000000000E
:1041700000000700000000006400000000000000D4
:0C41800040420F00FE2A0100D2040000A3
:00000001FF
